:020000040800F2
:10000000983900209D010008AF1100082D0F00084D
:10001000AB110008ED0C00085B3400080000000084
:1000200000000000000000000000000005010008C2
:10003000F10C00080000000049010008A92A00088E
:10004000B7010008B7010008B7010008051F000844
:10005000B7010008B7010008B7010008B7010008A0
:10006000B7010008B7010008B7010008B701000890
:10007000B7010008B7010008B7010008B701000880
:10008000B7010008B7010008B7010008B701000870
:10009000B7010008B7010008B7010008B701000860
:1000A000B7010008B7010008B7010008B701000850
:1000B000B7010008752B0008FD2B0008B7010008E8
:1000C000B7010008B7010008B7010008B701000830
:1000D000B70100081131000851310008B7010008CC
:1000E000B7010008B7010008B7010008DFF810D019
:1000F00000F088FC00480047C5400008AFF30080CE
:1001000098390020224B19680868B0E8F00F80F396
:100110000988BFF36F8F4FF0000080F311884EF015
:100120000D0E70470000000006480068006880F36C
:10013000088862B661B6BFF34F8FBFF36F8F00DFE1
:1001400000BF00BF08ED00E0EFF30980BFF36F8F41
:100150000F4B1A6820E9F00F106008B54FF05000FF
:1001600080F31188BFF34F8FBFF36F8F05F0BAFA9A
:100170004FF0000080F31188BDE808401968086856
:10018000B0E8F00F80F30988BFF36F8F704700BFAE
:10019000F0000020EFF3058070470000064880471C
:1001A00006480047FEE7FEE7FEE7FEE7FEE7FEE75C
:1001B000FEE7FEE7FEE7FEE7152B0008ED0000086E
:1001C00040EA01039B0703D009E008C9121F08C0D9
:1001D000042AFAD203E011F8013B00F8013B521E59
:1001E000F9D27047F0B480EA0102D40F4200B2EBBA
:1001F000410F02D20246084611464A0042D0C30DC2
:10020000DDB2C1F3C752AD1A202D35DAC1F31601A4
:1002100041F4000204B15242C5F1200602FA06F18F
:100220002A411044B3EBD05F23D0C4B1012DA0EB21
:10023000C35009DCF0BC4FF0004202EAC352DBB20B
:1002400000F5000000F03BBB400000F1807000EBC7
:10025000C350A0F1807040EAD170490009E049081C
:1002600041EAC071A0EBC35000F50000400800EB6C
:10027000C350F0BC00F01ABB6142012202EB410105
:10028000001BF6E7F0BC704781F00041AAE780F060
:100290000040A7E780EA010210B502F000434000E9
:1002A00022D04A001FD0010E01EB1261C0F35600AC
:1002B000C2F3560240F4000042F40002A0FB022008
:1002C00000047F39140400D0401C50EA124001D4CD
:1002D0004000491EC2B20C0604EBD010401C40087E
:1002E000802A02D003E0002010BD20F00100002988
:1002F00000DA0020184310BD30B480EA010202F099
:10030000004530F0004221F0004013D090B1C30D01
:10031000D40DC2F31601C0F31600E41A41F4000133
:1003200040F400027D34914201D3641C00E0490096
:10033000002C02DA30BC002070474FF4000000238C
:10034000914201D3891A034340084FEA4101F7D192
:1003500051B1914202D14FF0004105E002D24FF07D
:10036000010101E06FF0010103EBC450284430BCEF
:1003700000F09CBA2DE9FE4F804681EA0300C00FD1
:100380000C46009021F0004123F00045B8EB02003C
:10039000A94105D24046214690461C460B460246DE
:1003A00023F00040104347D0270DC7F30A00C3F3E2
:1003B0000A510290401A019040286BDAC3F31300EF
:1003C00040F4801B0098924620B10023D2EB030A30
:1003D00063EB0B0B01985946C0F14002504600F008
:1003E00034FA06460D4650465946019A00F04CFA3A
:1003F00010EB08006141002487EA115284EAE77398
:100400001A4340D0009A62B3019A012A4FEA075278
:1004100015DC001B61EB02014FF0004202EA0752BB
:10042000CDE90042001C41F5801132462B4600F018
:1004300083FA03B0BDE8F08F40462146F9E7001B80
:1004400061EB0201001C41F5801300185B4120188C
:10045000A2F5001747EB030140EAD570B6196D41CC
:1004600011E06D084FEA360645EAC0754FEA0752BB
:10047000001B61EB0201001C41F5801149084FEAA5
:1004800030000019514132462B4603B0BDE8F04F11
:1004900000F043BA0098012240000023D0EB020292
:1004A00063EBE073009821464FEAE074B8EB00007C
:1004B00061EB0401E9E783F000435BE781F0004171
:1004C00058E72DE9FE4F81EA030404F0004421F0CF
:1004D000004100944FF0000B23F0004350EA010468
:1004E0005ED052EA03045BD0C3F30A54C1F30A5549
:1004F0002C44A4F2F3340194A0FB0254C1F3130181
:1005000041F48011C3F3130343F4801301FB02444D
:1005100000FB034E840A970A44EA815447EA835752
:10052000A4FB076802958D0A05FB07854FEA932C0B
:1005300004FB0C542705029D4FEA065847EA16377C
:10054000B5EB08056EEB070C870E920E47EA811794
:1005500042EA8312A7FB0201B6EB0B0164EB000435
:100560002B0D43EA0C335E1844EB1C50DA4651461F
:10057000E7FB0201C5F313044FEA0B3343EA1453BC
:100580004FEA0432019C43EA0603A4F10C040294EE
:10059000009CCDE900B400F0CFF903B0BDE8F08FC6
:1005A00000200146F9E72DE9F04D81EA030404F04B
:1005B000004B21F0004514464FF0000A23F00041A3
:1005C00050EA050220D054EA01021DD0C5F30A57B3
:1005D0000246C5F31303C1F31300C1F30A5640F4F6
:1005E000801543F48013A7EB0608101BD64608F2CB
:1005F000FD3873EB050002D308F1010801E0921801
:100600005B41B8F1000F03DA00200146BDE8F08D30
:1006100000204FF48011064684460EE0171B73EB52
:10062000050705D3121B63EB050306434CEA010CD7
:1006300049084FEA300092185B4150EA0107EDD1BA
:1006400052EA030012D082EA040083EA050108435B
:1006500005D0101BAB4106D20122002306E0002288
:100660004FF0004302E06FF0010253101AEB060056
:100670004CEB085110EB0A0041EB0B01BDE8F04DCB
:1006800000F04BB9C10F80EAE0700844CA07962316
:10069000002100F014B90EB5C10F80EAE0700844E3
:1006A000CA07002140F233438DE80E000A460B468C
:1006B00000F042F903B000BD0EB540F233410291A3
:1006C0000021CDE900110A460B4600F035F903B0D0
:1006D00000BD20F00040C10DC0F3160040F4000042
:1006E0007F2901DA00207047962903DCC1F19601C9
:1006F000C8407047963988407047C1F30A5210B518
:10070000C1F3130140F2FF3341F480119A4201DA40
:10071000002010BD40F233439A42A2F2334203DC80
:10072000524200F0A1F810BD904010BD30B5041E3B
:1007300071F1000404DB4FF00044404264EB01011E
:10074000141E73F1000405DB1C464FF000435242B7
:1007500063EB0403994208BF904230BD01F00043AF
:1007600030B421F0004150EA010206D00A0DA2F592
:100770006072C1F31301002A02DC30BC0020704714
:10078000440F44EAC104C100E01830BC00EBC25081
:1007900000F08CB8002801DBC0F10040002901DB2B
:1007A000C1F1004181427047002801DBC0F10040E7
:1007B000002901DBC1F100418842704730B50B468A
:1007C000014600202022012409E021FA02F59D4281
:1007D00005D303FA02F5491B04FA02F52844151E55
:1007E000A2F10102F1DC30BD2DE9F05F05460020E9
:1007F00092469B4688460646814640241BE0284692
:1008000041464746224600F02FF853465A46C01A42
:10081000914110D311461846224600F016F82D1AC1
:1008200067EB01084F4622460120002100F00DF839
:1008300017EB00094E41201EA4F10104DFDC4846FD
:1008400031462A464346BDE8F09F202A04DB203A81
:1008500000FA02F1002070479140C2F1200320FA13
:1008600003F3194390407047202A04DB203A21FA11
:1008700002F00021704721FA02F3D040C2F12002B9
:100880009140084319467047202A06DBCB17203ACF
:1008900041FA02F043EAE07306E041FA02F3D04085
:1008A000C2F1200291400843194670470029A8BFB1
:1008B0007047401C490008BF20F00100704710B489
:1008C000B0FA80FC00FA0CF050EA010404BF10BC3E
:1008D000704749B1CCF1200421FA04F411FA0CF16B
:1008E00018BF012121430843A3EB0C01CB1D4FEAA4
:1008F00000614FEA102042BF002010BC704700EB9F
:10090000C35010440029A4BF10BC7047401C4900CC
:1009100008BF20F0010010BC704710B5141E73F121
:10092000000408DA401C41F1000192185B411A43AF
:1009300001D120F0010010BD2DE9F04D92469B46FB
:1009400011B1B1FA81F202E0B0FA80F220329046A1
:10095000FFF77BFF04460F4640EA0A0041EA0B011D
:1009600053465A46084313D0114653EA010019D0A2
:10097000C8F140025046FFF777FF05460E46504645
:1009800059464246FFF761FF084305D0012004E0C5
:1009900020463946BDE8F08D0020054346EAE07662
:1009A0002C4337430A986305E40AA0EB08000022B1
:1009B000FD0A44EA47540A3002D500200146E9E71F
:1009C000010510196941DDE9084500196941BDE8D3
:1009D000F04DA2E7C1F30A52C1F3130140F2FF3315
:1009E00041F480119A4202DA00200146704740F239
:1009F00033439A42A2F2334202DC5242FFF734BF41
:100A0000FFF723BF064C074D06E0E06840F0010306
:100A100094E8070098471034AC42F6D3FFF76AFB1E
:100A20004C6700086C67000870B58C1810F8015B03
:100A300015F0070301D110F8013B2A1106D110F877
:100A4000012B03E010F8016B01F8016B5B1EF9D17B
:100A50002B0705D40023521E0DD401F8013BFAE701
:100A600010F8013BCB1A921C03E013F8015B01F86C
:100A7000015B521EF9D5A142D8D3002070BD000001
:100A800070B5D378037013790B800B88022B08D1D3
:100A9000547903785B1E03EBC3035B00DB1C154D2D
:100AA000EC540B88032B08D1547903785B1E03EBBD
:100AB000C3035B001B1D0F4DEC540B88042B17DB8D
:100AC0000B88082B14DC55790B885B00DB1E04783F
:100AD000641E122606FB0433064CE55495790B88F8
:100AE0005B009B1E0478641E06FB0433014CE55436
:100AF00070BD00001C0000202DE9F04307ACF0CCD5
:100B000090F800C0ACF1010C0CEBCC0C4FEA4C0C93
:100B10000CF1030CDFF84C8118F80CC081F800C010
:100B200090F800C0ACF1010C0CEBCC0C4FEA4C0C73
:100B30000CF1040C18F80CC082F800C090F800C04A
:100B4000ACF1010C0CEBCC0C4FEA4C0C0CF1060C8C
:100B500018F80C8090F800C0ACF1010C0CEBCC0C38
:100B60004FEA4C0C0CF1050CDFF8F89019F80CC0AA
:100B700048EA0C2CA3F800C090F800C0ACF1010CBE
:100B80000CEBCC0C4FEA4C0C0CF1080CC84618F8D6
:100B90000C8090F800C0ACF1010C0CEBCC0C4FEACF
:100BA0004C0C0CF1070C19F80CC048EA0C2CA4F8FA
:100BB00000C090F800C0ACF1010C0CEBCC0C4FEA7B
:100BC0004C0C0CF10A0CC84618F80C8090F800C0C8
:100BD000ACF1010C0CEBCC0C4FEA4C0C0CF1090CF9
:100BE00019F80CC048EA0C2CA5F800C090F800C019
:100BF000ACF1010C0CEBCC0C4FEA4C0C0CF10C0CD6
:100C0000C84618F80C8090F800C0ACF1010C0CEB51
:100C1000CC0C4FEA4C0C0CF10B0C19F80CC048EA48
:100C20000C2CA6F800C090F800C0ACF1010C0CEB45
:100C3000CC0C4FEA4C0C0CF10E0CC84618F80C808A
:100C400090F800C0ACF1010C0CEBCC0C4FEA4C0C52
:100C50000CF10D0C19F80CC048EA0C2CA7F800C0D8
:100C6000BDE8F0831C00002010B5012000F0E8FC76
:100C7000002000F0E5FC10BD08B501460020009002
:100C8000034800900098084400900098008808BD30
:100C9000006C0040014908607047000000860D426A
:100CA00008B500220092044A0092009A0244009281
:100CB000009A116008BD0000006C004070B502464B
:100CC000CB781370042000BF0AE00D5C431E14783B
:100CD000641E122606FB0433034CE554431CD8B2B1
:100CE0001028F2DB70BD00001C00002000BFFEE7F2
:100CF00070472DE9F0410246002500260020002320
:100D00000024002791F803C00CF00F0591F803C0F0
:100D10000CF0100CBCF1000F03D091F802C04CEAAB
:100D2000050591F800C0BCF1000F31D01468002017
:100D30002BE04FF0010C0CFA00F3B1F800C00CEA04
:100D400003069E4220D183004FF00F0C0CFA03F7EC
:100D5000BC4305FA03FC4CEA040491F803C0BCF15F
:100D6000280F06D14FF0010C0CFA00FCC2F814C099
:100D70000AE091F803C0BCF1480F05D14FF0010C17
:100D80000CFA00FCC2F810C0401C0828D1D3146033
:100D9000B1F800C0BCF1FF0F34DD546800202EE034
:100DA00000F1080C4FF0010808FA0CF3B1F800C08C
:100DB0000CEA03069E4221D183004FF00F0C0CFA7F
:100DC00003F7BC4305FA03FC4CEA040491F803C0A2
:100DD000BCF1280F05D100F1080C08FA0CF8C2F894
:100DE000148091F803C0BCF1480F07D100F1080C42
:100DF0004FF0010808FA0CF8C2F81080401C0828CF
:100E0000CED35460BDE8F081416170470161704705
:100E100070B50C46FF2515701D700CE010F8015BD5
:100E2000167885EA06011D78064E765C75401570C9
:100E3000054D6D5C1D70251EA4F10106B4B2EDD107
:100E400070BD0000346500083466000808B5012153
:100E5000112000F0D5FB012000F0BCFB002000F0C9
:100E6000A3FC0020FFF716FF4FF46040ADF8000030
:100E700002208DF8020010208DF803006946064814
:100E8000FFF737FF002000F0A5FB4FF46041024858
:100E9000FFF7BCFF08BD00000010014010B504467C
:100EA00001200D4908600D49C1F8B801204600F045
:100EB00017F800200849091F0860022003F098F87D
:100EC00001200649C1F8B801022003F091F8002082
:100ED0000149091F086010BDBC01224200002242E6
:100EE00070B50446002500BF18E004F0800018B17A
:100EF00001200C49086002E000200A490860002037
:100F0000084908310860052003F052F8012006491D
:100F1000C1F8BC016006040E681CC5B2082DE4DBF4
:100F200070BD0000B40122420000224200BFFEE773
:100F30001FB55B480078EE2868D159484078B6283C
:100F400064D15748807803281BD1554A55495648E3
:100F5000FFF796FD55A002F0B9FB5A485A495B4A83
:100F60005B4BCDE90032CDE902105A4B5A4A5B493E
:100F70005B48FFF7C1FD02F089FB0B21002001F067
:100F800065F947488078042821D14548C0785549FB
:100F9000087055A002F09AFB002000900346012241
:100FA0000921019040F2E77001F0ECF84D4800781B
:100FB0004B4908704B4800785249087002F066FBB4
:100FC0000821002001F042F9802001F037F934486F
:100FD000807801281AD132493348FFF76FFE324832
:100FE000017849A002F072FB36483749374A384B3E
:100FF000CDE90032CDE90210364B374A374938483F
:10100000FFF77AFD1421002001F020F92448007830
:10101000EE2843D122484078B1283FD1204880783B
:1010200011280BD11E48C07BFF2807D13C48007C0B
:10103000FF2803D11121002001F008F91848807819
:1010400011280BD11648807BFF2807D13448C07B7C
:10105000FF2803D11021002001F0F8F81048807813
:1010600011280BD10E48007BFF2807D10C48407B8C
:10107000FF2803D10E21002001F0E8F8084880780D
:1010800001280BD10648C079FF2807D10448007A0F
:10109000FF2803D10921002001F0D8F81FBD00006E
:1010A0000C3400207C0500207A05002042362030D8
:1010B0003320636D643A2062617463682073796ED3
:1010C000630D0A00900500208E0500208C0500208D
:1010D0008A05002088050020930500209205002045
:1010E0008705002094050020423620303420636DAF
:1010F000643A206368616E67652073746167650D8B
:101100000A00000072050020423620303120636D55
:10111000643A20676574206F6E652025640D0A00AF
:10112000E00600204CF6CC40014908607047000002
:101130000030004010B500F001F810BD4AF6AA20BA
:1011400001490860704700000030004001494860D4
:10115000704700000030004001498860704700007F
:101160000030004001490860704700000030004036
:101170000146CA1701EB92729210A1EB820292B95A
:10118000642091FBF0F200FB121050B94FF4C870CC
:1011900091FBF0F200FB121008B90120704700200B
:1011A000FCE70120FAE70020F8E700BFFEE7704700
:1011B00070B5002100230F22C47804B3154C2468B5
:1011C00004F4E064C4F5E064210AC1F10403CA40F8
:1011D000447804FA03F184781440214309010E4C49
:1011E0000678A155047804F01F050124AC40057869
:1011F0006D11AD0005F1E025C5F8004109E0047866
:1012000004F01F050124AC40044D0678761145F822
:10121000264070BD0CED00E000E400E080E100E05D
:1012200002490143024A1160704700000000FA05BC
:101230000CED00E070B55648806B5549C96888428E
:1012400000DA70BD524948684FF07E51FEF7CAFF80
:1012500006464F4801683046FFF79CFA0BD24D49CD
:10126000097801F0FB014B4A11700846FFF716FEA2
:10127000022049490870464908684FF07E51FEF740
:10128000B1FF0646424841683046FFF783FA0BD269
:101290004049097841F004013E4A11700846FFF7C1
:1012A000FDFD01203C490870394A51681068FFF77C
:1012B0007BFA07D2364A51681068FEF7E5FF3449D9
:1012C000886106E0324A11685068FEF7DDFF304958
:1012D00088612F4A91699068FEF7DCFF2C4988628B
:1012E0000A469169106AFEF77DFF294908620A469D
:1012F000D1699069FEF7C8FF05462548016A27486D
:101300000068FEF7C7FF2249486229462448006862
:10131000FEF7C0FF1E49C862C86A0021FFF73AFA0B
:1013200006D21B48C16A0020FEF7AEFF1849C8620A
:10133000174A516A906AFEF755FF06461448C16A7B
:101340003046FEF74FFF04461149C86BFFF79AF984
:1013500006462146FFF71EFA06D20D49C86BFFF775
:1013600091F90B4948630BE000212046FFF712FA80
:1013700004D80748006B0649486301E00448446309
:10138000034880690249C8610020886300BF58E7AC
:101390006C0700207805002080050020CC0000208C
:1013A000D00000200648074988604FF4FA70C860F2
:1013B000C820C8634FF07E500863002088637047E0
:1013C00000002A436C07002030B589B005460C4662
:1013D0000121C80200F014F90121042000F010F9E5
:1013E00018208DF823004FF48070ADF82000032002
:1013F0008DF8220008A91B48FFF77BFC0020ADF800
:101400001A00ADF81600ADF81850ADF814408DF87C
:101410001C0005A9144801F0E5FD01A801F0CFFD6D
:101420006020ADF804000020ADF80C000120ADF8FC
:1014300006000020ADF80A0001A90B4801F072FC7B
:101440000121094801F045FC0821074801F0B6FCDC
:101450000121054801F022FC0121034801F02DFC87
:1014600009B030BD00080140002C014030B589B002
:1014700005460C460121C80200F0C2F801210420F3
:1014800000F0BEF818208DF823004FF40060ADF88E
:10149000200003208DF8220008A91B48FFF729FC33
:1014A0000020ADF81A00ADF81600ADF81850ADF8F0
:1014B00014408DF81C0005A9144801F093FD01A803
:1014C00001F07DFD6020ADF804000020ADF80C00B7
:1014D0000120ADF806000020ADF80A0001A90B4874
:1014E00001F022FD0121094801F0F3FB0821074822
:1014F00001F058FD0121054801F0D0FB012103480E
:1015000001F0DBFB09B030BD00080140002C0140B8
:1015100030B589B005460C460121084600F060F858
:101520000121042000F06CF818208DF8230002201F
:10153000ADF8200003208DF8220008A91648FFF717
:10154000D8FB0020ADF81A00ADF81600ADF8185021
:10155000ADF814408DF81C0005A94FF0804001F053
:1015600041FD01A801F02BFD6020ADF80400002032
:10157000ADF80C000120ADF806000020ADF80A001F
:1015800001A94FF0804001F023FC0121880701F000
:1015900094FB09B030BD00000008014010B50446BE
:1015A0002146024801F015FD10BD0000002C01404D
:1015B00010B5044621464FF0804001F00CFD10BDEF
:1015C00010B504462146024801F009FD10BD000097
:1015D000002C0140014908627047000000000E42E3
:1015E00029B1064AD2690243044BDA6104E0034A96
:1015F000D2698243014BDA6170470000001002405B
:1016000029B1064A92690243044B9A6104E0034AF5
:1016100092698243014B9A617047000000100240BA
:1016200029B1064AD2680243044BDA6004E0034A57
:10163000D2688243014BDA6070470000001002401C
:1016400001490860704700004004424230B5002163
:101650000022002400232D4D6D6805F00C0121B1FE
:10166000042905D0082923D105E0294D056022E091
:10167000274D05601FE0254D6D6805F47012234D60
:101680006D6805F48034022505EB92421CB9214DAA
:10169000554305600BE01D4D6D6805F400351DB127
:1016A0001C4D5543056002E0194D5543056002E0AD
:1016B000174D056000BF00BF144D6D6805F0F001C7
:1016C0000909154D6B5C0568DD4045600F4D6D687F
:1016D00005F4E061090A104D6B5C4568DD408560EA
:1016E0000A4D6D6805F46051C90A0B4D6B5C456885
:1016F000DD40C560054D6D6805F44041890B074D1F
:101700006B5CC568B5FBF3F5056130BD00100240A8
:1017100000127A0000093D00DA000020EA000020F3
:1017200010B501460022002300204A11012A02D1EF
:10173000094C236806E0022A02D1074C236A01E023
:10174000054C636A01F01F02012494401C400CB157
:10175000012000E0002010BD00100240114909687E
:1017600021F480310F4A11601146096821F480216B
:101770001160B0F5803F03D0B0F5802F0ED106E0A8
:101780000849096841F48031064A116007E00549BB
:10179000096841F4A021034A116000E000BF00BFC6
:1017A000704700000010024000210B4A11700A4AE5
:1017B000203A82F82010012802D0042808D103E042
:1017C0000121054A117004E00521034A117000E06F
:1017D00000BF00BF704700002010024001490860B0
:1017E000704700003C0442420249096A0143014A31
:1017F000116270470010024010B586B0044600F038
:101800006BFD20213348FFF7FFFA40213148FFF7F5
:10181000FDFA01210C20FFF7F3FE01218803FFF7F9
:10182000EFFE4FF40060ADF8140010208DF81700A3
:1018300003208DF8160005A92648FFF75AFA4FF441
:101840000070ADF8140018208DF8170005A9224883
:10185000FFF74FFA4FF48060ADF8140004208DF8C4
:10186000170005A91C48FFF744FA01218803FFF778
:10187000D7FE00214FF48040FFF7D2FE01940020F4
:10188000ADF80800ADF80A00ADF80C00ADF8100096
:101890000C20ADF80E0001A9104801F069FD2520CB
:1018A0008DF8000000208DF8010001208DF8030064
:1018B0006846FFF77DFC012240F22551074801F000
:1018C00032FD0121054801F0EBFC002004490860CD
:1018D00006B010BD000C0140000801400038014076
:1018E000AC81214270B505460E4601200E490860C4
:1018F00000240CE000BF40210C4801F0DDFC002872
:10190000F9D0295D094801F0A4FD601CC4B2B442BD
:10191000F0DB00BF4021054801F0CEFC0028F9D0E3
:1019200000200149086070BDAC81214200380140AF
:1019300010B5EE20B4490870B520487005208870B5
:10194000FF204876FC208876FF20C87608770120A3
:10195000AE490860AE480068B0F5FA7F07DCAD48D4
:10196000C078AD490870AB480079AC490870AC4804
:101970000068B0F57A7F07DCA6484079A94908706D
:10198000A4488079A8490870A34800789E49C87087
:10199000A24800780871A34800784871A2480078EE
:1019A0008871A2480078401E00EBC00040000A3059
:1019B0009F49095C9D480078401E00EBC000400034
:1019C00009309B4A105C41EA00209A4908809748F8
:1019D0000078401E00EBC00040000C301146095C4E
:1019E00092480078401E00EBC00040000B30105CB5
:1019F00041EA0020904908808C480078401E00EBA6
:101A0000C00040000E301146095C88480078401E36
:101A100000EBC00040000D30105C41EA0020874917
:101A2000088084480088B0F57A7F15DC7F4800780C
:101A3000401E00EBC000400009301146085C8049A0
:101A400008707A480078401E00EBC00040000A3061
:101A50001146085C7B49087077480088B0F57A7FAA
:101A600015DC72480078401E00EBC00040000B30CF
:101A70006F49085C744908706C480078401E00EBA0
:101A8000C00040000C306A49085C704908706B481F
:101A90000088B0F57A7F15DC64480078401E00EBC2
:101AA000C00040000D306249085C694908705F4819
:101AB0000078401E00EBC00040000E305C49085C1E
:101AC000644908705E4800784F49C8715D480078E5
:101AD00008725D48007848725C48007888725C48FB
:101AE0000078C8725B48007808735B48006841F270
:101AF0008831884207DC4748C07C5849087045480F
:101B0000007D57490870554800783F49487354484C
:101B1000007888734548007807283CDA4348007805
:101B2000401E00EBC0004000C01C4149085C182862
:101B300031DA3E480078401E00EBC0004000001D36
:101B4000085C3C2827DA47480078182823DA4648FA
:101B500000783C281FDA354800782B49C873334891
:101B60000078401E00EBC0004000C01C3049085CFB
:101B7000254908742D480078401E00EBC000400045
:101B8000001D2B49085C2049487436480078887449
:101B900035480078C874354800781B4908753448C2
:101BA0000078487533480078887517230322324837
:101BB00002F0F1F9314B324A14212F48FFF728F98E
:101BC0002F4800781049C8752C4800780876002402
:101BD0000DE000BF40212B4801F06EFB0028F9D03A
:101BE0000948015D274801F034FC601CC4B21D2C7B
:101BF000EFDB00BF4021234801F05EFB0028F9D055
:101C000000200249086010BD88000020AC812142FC
:101C1000A00500200C340020A5000020A600002014
:101C2000A4050020A7000020A800002087050020B0
:101C30001C000020AC000020B0000020AE000020FE
:101C4000B2000020B3000020B6000020B700002042
:101C5000B4000020B5000020A8050020A900002045
:101C6000AA0000207E0500207F05002080050020BE
:101C70008105002082050020CC060020B90000204C
:101C8000B8000020003801401CB519A103C9CDE9F6
:101C90000001012018490860184800788DF80300F9
:101CA00016480078401C1549087008460078062838
:101CB00001DD0120087000240DE000BF4021104824
:101CC00001F0FAFA0028F9D01DF804100C4801F0D0
:101CD000C0FB601CC4B2082CEFDB00BF40210848E9
:101CE00001F0EAFA0028F9D00020034908601CBD81
:101CF000EEB50100FFFCFFFFAC8121427905002019
:101D000000380140024909888143014A1180704727
:101D1000042800400348008840F010000149088072
:101D20007047000004280040034800884FF6EF7118
:101D30000840014908807047042800402DE9F0411F
:101D400006460F464FF000080024002500F082F8F8
:101D500080463C48B8FBF0F43B480088A0423CD0A9
:101D600039490C8040F2B27510E02846FFF700FABE
:101D700040B1B4F5B77F02D3A4F5B77404E0681C92
:101D800085B206E0A4F26D14681C85B2B4F5B67F86
:101D9000EBD800BF2D488580002516E02B498888A8
:101DA000FFF7E6F930B1012D04D11D2C01D31D3C04
:101DB00009E00CE02648405DA04203D82448405D7D
:101DC000241A00E003E0681C85B21C2CE6D200BF98
:101DD000681C1E498871601CC8711A48B8FBF0F174
:101DE00000FB11844FF46160B4FBF0F017490870F8
:101DF0004FF46160B4FBF0F100FB11403C21B0FBFB
:101E0000F1F0124948704FF46160B4FBF0F100FB4F
:101E100011403C21B0FBF1F201FB12000B4988702C
:101E20000B46DA799979988800F030F807490872FA
:101E30000846007830700846407838700020BDE8C9
:101E4000F081000080510100BE00002060070020EA
:101E500040670008002103480188001F008841EA0C
:101E6000004070471C28004001460020064A1288A6
:101E70000A40D0B2044A121F12880A4012B108B1B7
:101E8000012000E00020704704280040F0B5034620
:101E90000C461546642093FBF0F0C6B2642093FB19
:101EA000F0F700FB1730C1B2132E02DD01F1640020
:101EB000C1B20846CF1701EB977701EBA707BAB27B
:101EC000072092FBF0F700FB172082B25719601E23
:101ED000DFF82CC01CF80000384482B2CF1701EBA9
:101EE0009777BF10A1EB87071FB9032C01DA501EAB
:101EF00082B2072092FBF0F700FB1720C0B2F0BDC2
:101F00003467000810B50120FFF7AEFF18B10A4989
:101F10000A48FFF713FF0220FFF7A6FF30B10220A7
:101F2000FFF7F0FE04490548FFF708FF0520FFF71B
:101F3000E9FE00F00BF910BDBD000020BC00002040
:101F400029B1064A12880243044B1A8004E0034A6E
:101F500012888243014B1A8070470000002800401D
:101F60001CB5002401214FF0C050FFF739FB0120C0
:101F7000FFF730FB0420FEF77FFE45F25001884258
:101F800040D0FEF771FE4FF48030FFF7E7FB04E02E
:101F9000601CC4B20A2002F00BF83120FFF7C0FB2E
:101FA00008B9FA2CF4DBFA2C01DB01201CBD4FF43C
:101FB0004070FFF719FC0120FFF710FC00F0C6F895
:101FC00000F0CEF801210846FFF7BAFF00F0BEF896
:101FD000FFF7A0FE4FF2244000F0A8F800F0B6F89A
:101FE00000200090034601220921019040F2E77091
:101FF00000F02AF8FFF798FE45F250010420FEF7A2
:102000004FFE07E000F0ACF801210846FFF798FF0B
:1020100000F09CF800F00AF802490348FFF78EFE32
:102020000020C3E7BD000020BC00002008B503204D
:102030008DF8000001208DF801008DF8030068463E
:10204000FFF7B6F808BD00002DE9F05F06460F4621
:1020500090469946DDE90AAB002440F2B270864210
:1020600003DB40F63300864202DD0120BDE8F09F2D
:1020700040F2B2750AE02846FFF77AF810B120481E
:10208000044401E01F480444681C85B2B542F2DBF9
:10209000781EC7B2002510E01B48405D40F2A32126
:1020A000484304EBC0143046FFF762F818B1012D25
:1020B00001D116480444681C85B2BD42ECDBA8F18E
:1020C000010040F2A321484304EBC014C9EB4910BE
:1020D000C0EB092004EB0014CAEB0A1004EB8004E7
:1020E0005C4401214FF0C050FFF77AFA0120FFF75E
:1020F00071FA204600F00CF800F028F80020B5E74F
:102100000085E2018033E101406700088051010051
:1021100000B50246FFF7FEFD100C03490880091DBB
:102120000A80FFF701FE00BD1828004000B50246F6
:10213000FFF7F0FDC2F3034003490880091D0A8040
:10214000FFF7F2FD00BD00000828004000BF034873
:10215000008800F020000028F9D0704704280040D3
:10216000074800884FF6F77108400549088000BF0E
:102170000348008800F008000028F9D070470000EC
:10218000042800402DE9FC4705460E4617469846B0
:10219000DDE90A9A002401214FF0C050FFF720FA30
:1021A0000120FFF717FAFEF75FFD4FF48030FFF7CD
:1021B000D5FA04E0601CC4B20A2001F0F9FE312017
:1021C000FFF7AEFA08B9FA2CF4DBFA2C02DB012097
:1021D000BDE8FC874FF44070FFF706FB0120FFF7D6
:1021E000FDFAFFF7B3FFFFF7BBFF01210846FFF73A
:1021F000A7FEFFF7ABFFFFF78DFD4FF22440FFF77F
:1022000095FFFFF7A3FF43463A4631462846CDE9FE
:10221000009AFFF719FFFFF787FD45F250010420F0
:10222000FEF73EFDFFF702FF02490348FFF786FD78
:102230000020CDE7BD000020BC000020002100BF31
:1022400000E0491C8142FCDB7047000010B50246EB
:102250000020104604E04318084CE35C2354401C63
:10226000C1F180038342F6DCC1F1800003E000236A
:10227000024C2354401C8028F9DB10BD0C34002094
:102280000146002003E00022024B1A54401C884201
:10229000F9DB70470C34002010B501F005F96C2211
:1022A0000021094801F028F96D230022064907485A
:1022B00001F071FE01226D21054801F01DF904486D
:1022C00000780449087010BDF40500201C000020AF
:1022D000160000208705002008B501210820FFF71F
:1022E0008FF9E020ADF8000010208DF803000320E6
:1022F0008DF8020069460448FEF7FBFC8021024885
:10230000FEF782FD08BD0000000C014000B587B05B
:1023100001210420FFF774F901210803FFF770F988
:10232000E020ADF8180018208DF81B0003208DF870
:102330001A0006A91748FEF7DCFCE0211548FEF755
:1023400065FD0020ADF804004FF48270ADF8060082
:102350000020ADF808000220ADF80A000120ADF819
:102360000C004002ADF80E003820ADF8100000203F
:10237000ADF812000720ADF8140001A9064800F0DE
:1023800067F80121044800F049F8FF2000F006F842
:1023900007B000BD000801400030014070B505469F
:1023A000002405E0601CC4B2C82C01DD002070BD13
:1023B00002210E4800F03EF80028F3D029460B48D1
:1023C00000F044F8002405E0601CC4B2C82C01DD14
:1023D0000020ECE70121054800F02CF80028F3D09C
:1023E000024800F030F8C0B2E1E7000000300140E0
:1023F00010B50446074800884FF6C77108400549E4
:10240000088008460088204308800121024800F027
:1024100005F810BD003800400030014021B10288AD
:1024200042F04002028004E002884FF6BF731A4077
:10243000028070470246002013890B400BB1012037
:1024400000E000207047014688897047818170470D
:1024500010B50022028802F441520B884C882343B5
:102460008C882343CC8823430C8923434C89234302
:102470008C892343CC8923431A430280838B4FF2F8
:10248000FF74234083830B8A038210BD1FB57BE258
:1024900002F010FDFB490870FB48FC49FC4AFD4B6B
:1024A000CDE90032CDE90210FB4BFC4AFC49F5486E
:1024B000FEF722FB0821FB48FFF714FAC82001F0C1
:1024C000BBFDFFF7E1FBC82001F0B6FD8023002231
:1024D000F549F64801F05FFD0020F54908707AE102
:1024E000F2480078012872D1F04840780328FAD1E8
:1024F000EE48C078EF490860EC480079096840EA86
:102500000120EC490860E9484079EB490860E74858
:102510008079096840EA0120E7490860E348C07C07
:10252000E6490860E148007D096840EA0120E34986
:102530000860E14800680A2190FBF1F201FB1204F7
:10254000DD48006890FBF1F5DA48006890FBF1F295
:1025500001FB1206D748006890FBF1F7D7480068E6
:102560002B4632463946CDE90040D5A001F0AEF801
:10257000C94800881438CF490968884214DCCD481E
:102580000168C5480088143081420DDCC1480088CC
:102590006438C9490968884206DCC7480168BD48F3
:1025A00000886430814213DDD048008840F2622107
:1025B00088420DDDCE49097841F00101CC4A117005
:1025C0000846FEF76BFC0120CA4908700CE0E5E004
:1025D000C749097801F0FE01C54A11700846FEF7A7
:1025E0005DFC0020C3490870B2480068B0F5167F52
:1025F00066DAB048006810F11E0F61DDBE48006861
:10260000AC490968401ABD490860084600680028BE
:1026100003DA0846006840420860B84800680328AA
:1026200003DBB548006800284AD19B480088FEF7C4
:1026300043F806460022B24BFDF7B5FF0446FEF70D
:102640008DF8B04908609B480068FEF724F80646FC
:102650000022AB4BFDF7A7FF0446FEF77FF8A94920
:102660004860FEF7E7FDA749C86BFEF70BF8064682
:10267000A449486BA449FDF70DFE07463146FDF716
:102680003BFE04464FF07E51FDF7FEFD0546FEF78A
:1026900020F89E49086008460068FEF70DF80546D8
:1026A0009B4A9C4BFDF70DFF0746FEF726F884B2C8
:1026B0002146994800F091FC7E4800688E490860E8
:1026C0007D480168734800883230814214DD8849B2
:1026D000097841F00801864A11700846FEF7DEFBD2
:1026E0008349097801F0EF01814A11700846FEF72D
:1026F000D5FB0120894908706648008832386E4948
:102700000968884214DD7A49097841F01001784A55
:1027100011700846FEF7C2FB7549097801F0F70110
:10272000734A11700846FEF7B9FB02207B49087016
:102730007A480078012811D15F4800685549098816
:1027400088420BDC6A49097801F0E701684A117098
:102750000846FEF7A3FB0020704908706F48007818
:10276000022811D1544800684A49098888420BDB85
:102770005F49097801F0E7015D4A11700846FEF7EC
:102780008DFB002065490870FFF7D2F81720FFF78E
:1027900077FD17210020FFF759FD1CE04348007822
:1027A000EE2802D1FEF7C4FB15E000243F48007874
:1027B00018B101210020FFF749FD00E0641C3B48EF
:1027C000005D0028FAD0E1B20020FFF73FFD54A0E1
:1027D00000F07CFF00BF8021344801F053FC00284A
:1027E0003FF47EAE354803683348026831480168DB
:1027F00051A000F06BFF26480088B0F57A7F40DCDE
:1028000022480088B0F57A7F3BDC21480088FDF73C
:1028100053FF824600224E4BFDF7C5FE8046002244
:102820004C4BFDF74EFE064600224B4BFDF7A2FD3A
:102830000446FDF762FF80B20390FEF7AFFE134837
:102840000088FDF739FF80460022414BFDF7ABFEC3
:10285000824600223F4BFDF734FE064600223E4BE7
:10286000FDF788FD0446FDF748FF80B20390FEF7B0
:102870009FFE05480088FDF71FFF06460022344BE7
:102880006CE07EE087050020900500208E0500208A
:102890008C0500208A050020880500209305002073
:1028A0009205002097050020E00600200C3400204F
:1028B000BA000020A0050020A4050020A8050020E3
:1028C0006E6F775F74656D3D25642E2564A1E62CDF
:1028D0006E6F775F68756D3D25642E256425252014
:1028E0002C636F323D25640D0A0000008405002032
:1028F0007805002082050020B00500207405002026
:10290000000024406C0700200000C843BC050020E4
:102910000AD7A3703D0AEB3F000400408105002068
:1029200070726576696F7573206172726179206368
:1029300075740D0A000000002564A3AC202020203F
:10294000256420A3AC202020202025640A0000005C
:102950000000594000000C4000003C40FDF723FE01
:1029600004460022094BFDF7ACFD80460022084BCF
:10297000FDF700FD8246FDF7C0FE80B20390FEF732
:102980001FFE00200349087082E5000000000C4093
:1029900000003C40BA00002010B500F001F810BD66
:1029A0000CB50020019000903348006840F480305E
:1029B0003149086000BF3048006800F400300090E2
:1029C0000198401C0190009818B90198B0F5A06FCB
:1029D000F1D12948006800F4003010B101200090C6
:1029E00001E0002000900098012843D123480068AE
:1029F00040F01000214908600846006820F00300FC
:102A000008600846006840F0020008601A48406804
:102A1000194948600846406848600846406840F4E4
:102A2000806048600846406820F47C104860084692
:102A3000406840F4E81048600846006840F0807044
:102A4000086000BF0C48006800F000700028F9D052
:102A50000948406820F0030007494860084640687C
:102A600040F00200486000BF0348406800F00C00DE
:102A70000828F9D10CBD00000010024000200240DF
:102A8000042808D14FF0E021096941F004014FF01A
:102A9000E022116107E04FF0E021096921F0040113
:102AA0004FF0E0221161704710B503F09DFA012844
:102AB00001D002F0BBFE10BD70B505460420FFF743
:102AC000DFFF104800681049B0FBF1F00F490870B3
:102AD0000C4800680C49B0FBF1F44FF47A704443A1
:102AE00001200B4908804FF0E020006940F002000F
:102AF0004FF0E021086108464461006940F00100A0
:102B0000086170BD0000002040420F00D40000208A
:102B1000D600002010B51348006840F001001149AC
:102B2000086008464068104908400E494860084659
:102B300000680E4908400B4908600846006820F408
:102B4000802008600846406820F4FE0048604FF48A
:102B50001F008860FFF720FF4FF000600449086005
:102B600010BD0000001002400000FFF8FFFFF6FE5D
:102B700008ED00E010B50121064800F0B9F840B1B9
:102B80000548806B401C044988630121014800F01E
:102B900091F810BD000400406C0700201FB5012112
:102BA0000220FEF71DFD1D208DF80C0003208DF87E
:102BB0000D0001208DF80F0003A8FEF7F9FA4FF47D
:102BC0007A70ADF804004720ADF800000020ADF8A1
:102BD00002006946084800F005FA0122114606483D
:102BE00000F097F80121044800F064F80121024840
:102BF00000F063F81FBD00000004004010B5012183
:102C00000D4800F075F8B0B101210B4800F052F802
:102C10000A480088401C0949088009480078401C7F
:102C20000749087008460078052804DDFEF782FA97
:102C300000200349087010BD0008004084050020F2
:102C4000860500207FB505460C4601210420FEF7CD
:102C5000C7FCADF80850ADF804400020ADF80A00FC
:102C6000ADF8060001A90C4800F0BCF9012211469C
:102C7000094800F04EF81E208DF8000002208DF863
:102C8000010001208DF803006846FEF791FA01214A
:102C9000014800F012F87FBD0008004021B1028811
:102CA00042F08002028004E002884FF67F731A40EF
:102CB00002807047CA430282704721B1028842F005
:102CC0000102028004E002884FF6FE731A4002807F
:102CD000704731B1B0F8442042F40042A0F84420DB
:102CE00005E0B0F84420C2F30E02A0F8442070477B
:102CF00030B50246002000230024158A05EA0103AE
:102D0000958905EA010413B10CB1012000E000200F
:102D100030BD1AB183890B43838102E083898B43E1
:102D20008381704770B5002400220023058C4FF684
:102D3000FE7635400584028C8388048B4FF68F75B0
:102D40002C40B51E2C400D882C43751E2A400D8941
:102D50002A434D882A43144DA8420BD0134DA84254
:102D600008D0134DA84205D0124DA84202D0124DF2
:102D7000A84213D14FF6F7752A404D892A434FF6E2
:102D8000FB752A408D882A434FF6FF652B404FF68E
:102D9000FF552B408D892B43CD892B4383800483A2
:102DA000CD888586028470BD002C0140003401402E
:102DB0000040014000440140004801400A46002113
:102DC000018B4FF6F77319401143018370470000E0
:102DD00070B5002400220023058C4FF6EF763540B5
:102DE0000584028C8388048B48F6FF752C404FF6CF
:102DF000FF452C400D884FF6FF7606EA05252C434B
:102E00004FF6DF752A400D8906EA05152A434D88DD
:102E100006EA05152A43154DA84202D0144DA842D2
:102E20001DD14FF67F752A404D894FF6FF7606EA91
:102E300005152A434FF6BF752A408D8806EA051509
:102E40002A434FF6FF352B404FF2FF752B408D89FB
:102E500006EA85052B43CD8906EA85052B43838049
:102E60000483CD880587028470BD0000002C0140DA
:102E70000034014070B5002400220023058C4FF679
:102E8000FF6635400584028C8388848B4FF68F75EE
:102E90002C404FF6FC752C400D882C434FF6FF5507
:102EA0002A400D894FF6FF7606EA05252A434D880C
:102EB00006EA05252A43154DA84202D0144DA84222
:102EC0001DD14FF2FF752A404D894FF6FF7606EA75
:102ED00005252A434FF6FF352A408D8806EA052549
:102EE0002A434EF6FF752B404DF6FF752B408D891A
:102EF00006EA05152B43CD8906EA05152B43838089
:102F00008483CD888587028470BD0000002C014039
:102F1000003401400A460021818B4FF6F7731940B7
:102F2000114381837047000070B500220023002404
:102F3000058C4EF6FF7635400584038C8488828BA1
:102F400048F6FF752A404FF6FF452A400D884FF698
:102F5000FF7606EA05252A434DF6FF752B400D89BD
:102F600006EA05352B434D8806EA05352B430B4D04
:102F7000A84202D00A4DA84208D14BF6FF752C405A
:102F80008D894FF6FF7606EA85152C43848082836F
:102F9000CD88A0F84050038470BD0000002C014093
:102FA000003401400A460021818B4FF2FF73194023
:102FB0004FF6FF7303EA0223194381837047002110
:102FC000018041808180C180018141818181C181F5
:102FD0007047818670470187704781877047A0F8E6
:102FE00040107047002202881D4B98420ED01D4BA6
:102FF00098420BD0B0F1804F08D01B4B984205D0BF
:103000001A4B984202D01A4B984204D14FF68F7354
:103010001A404B881A43174B984207D0164B9842D8
:1030200004D04FF6FF431A40CB881A4302808B88A6
:1030300083850B8803850A4B98420BD0094B984235
:1030400008D00E4B984205D00D4B984202D00D4B44
:10305000984201D10B7A03860123838270470000D6
:10306000002C0140003401400004004000080040F2
:10307000000C0040001000400014004000400140DF
:10308000004401400048014030B589B005460C4677
:1030900001210920FEF7B4FA0120ADF82000182024
:1030A0008DF8230003208DF8220008A91648FDF7AB
:1030B00020FE01210220FEF793FAA8B2ADF8180015
:1030C000A0B2ADF814000020ADF81A00ADF816005B
:1030D00005A90E48FFF786FF7020ADF80400012017
:1030E000ADF806000220ADF80C0001A90748FFF773
:1030F000C1FE08210548FFF70DFF01210348FFF736
:10310000DCFD09B030BD0000000C014000040040AF
:1031100010B540F225510B4800F0DBF880B10948AA
:1031200000F092F9C4B208480078802808DA07480D
:1031300005490978445404480078401C0249087045
:1031400010BD000000380140BA000020E006002059
:1031500010B540F225511D4800F0BBF810B31B48D4
:1031600000F072F9C4B21A48008800F40040C8B9EF
:103170001748008800F4804060B10A2C03D000207A
:103180001349088020E01248008840F400401049AC
:10319000088019E00D2C06D10D48008840F48040CD
:1031A0000B49088010E00A480088C0F30D00094967
:1031B0000C5407480088401C0549088008460088D0
:1031C000FE2801DD0020088010BD00000044004002
:1031D000D8000020B007002010B586B004460121B9
:1031E0004804FEF7FDF901210C20FEF709FA4FF41F
:1031F0000070ADF8140003208DF8160010208DF833
:10320000170005A92248FDF774FD0420ADF814004D
:1032100003208DF8160018208DF8170005A91D4809
:10322000FDF767FD0820ADF8140004208DF81700A5
:1032300005A91848FDF75DFD26208DF80000042043
:103240008DF8010001208DF803006846FDF7B0FFFE
:1032500001940020ADF80800ADF80A00ADF80C00AC
:10326000ADF810000C20ADF80E0001A90A4800F0DE
:103270007FF8012240F22551074800F054F801215F
:10328000054800F00DF800200449086006B010BDA4
:10329000000C01400008014000440040A48121428C
:1032A00021B1828942F40052828104E082894DF684
:1032B000FF731A408281704702460020B1F5007FFB
:1032C00000D100BF13880B400BB1012000E00020AB
:1032D000704770B50246002400230025002040F608
:1032E0006A16B14200D100BFC1F3421501F01F03BD
:1032F000012606FA03F3012D02D19689334006E038
:10330000022D02D1168A334001E0968A33400C1216
:10331000012606FA04F41688344013B10CB10120DA
:1033200000E0002070BDF0B5034600240026002513
:10333000002040F66A17B94200D100BF1846C1F319
:10334000421401F01F06012707FA06F5012C01D1EE
:103350000C3004E0022C01D1103000E014301AB11E
:1033600007682F43076002E00768AF430760F0BDBE
:103370002DE9F04786B005460E460024A24600BF60
:10338000A1460027B08900B100BF2F462C8A4CF619
:10339000FF700440F08804432C82AC894EF6F31091
:1033A0000440B08831890843718908430443AC81E3
:1033B000AC8A4FF6FF400440B0890443AC8201A8B8
:1033C000FEF744F91F48874202D1DDF810A001E062
:1033D000DDF80CA0A88900F4004040B10AEBCA0057
:1033E00000EB0A1031684900B0FBF1F807E00AEB86
:1033F000CA0000EB0A1031688900B0FBF1F86420C4
:10340000B8FBF0F004012009642101FB1089A889B0
:1034100000F4004040B1322000EBC900B0FBF1F0F5
:1034200000F00700044308E0322000EB091064219B
:10343000B0FBF1F000F00F0004432C8106B0BDE8B2
:10344000F08700000038014001468888C0F308007A
:103450007047C1F308028280704700BFFEE700009A
:1034600010B50446240300F0B3F800F0A7F80020DC
:103470000B4908602020FEF791FFC4F30740FEF7D8
:103480008DFFC4F30720FEF789FFE0B2FEF786FF49
:1034900001200449C1F8900100F090F810BD00002F
:1034A000900121420000214208B501210420FEF7CD
:1034B000A7F81020ADF800008DF8030003208DF868
:1034C000020069460948FDF714FC10210748FDF782
:1034D0009DFC012006490860FEF718FF0020FEF75A
:1034E00087FF00F031F80349088008BD000801405B
:1034F00090012142140000202DE9F04106460C46BF
:10350000174600200F4908600320FEF747FFC4F369
:103510000740FEF743FFC4F30720FEF73FFFE0B28A
:10352000FEF73CFF002505E0FF20FEF737FF705552
:10353000681C85B2BD42F7DB012002490860BDE886
:10354000F08100009001214210B5002400200E49B6
:1035500008609020FEF722FF0020FEF71FFF0020EA
:10356000FEF71CFF0020FEF719FFFF20FEF716FFF5
:1035700044EA0024FF20FEF711FF04430120034921
:10358000C1F89001204610BD900121420000214267
:1035900010B500240020074908600520FEF7FEFE54
:1035A000FF20FEF7FBFE044601200349C1F890010D
:1035B000204610BD900121420000214210B500BFFD
:1035C000FFF7E6FF00F001000028F9D110BD000070
:1035D00010B50020044908600620FEF7DFFE012038
:1035E0000249C1F8900110BD900121420000214222
:1035F0002DE9F04107460E461446F0B2C0F580753D
:10360000AC4200DC254612E02A463146384600F03E
:1036100013F8AC4200D10BE02F442E44601B84B25F
:10362000B4F5807F02DD4FF4807500E02546EBE7BE
:1036300000BFBDE8F08100002DE9F04106460C46D0
:103640001746FFF7C5FF00200F4908600220FEF76C
:10365000A5FEC4F30740FEF7A1FEC4F30720FEF762
:103660009DFEE0B2FEF79AFE002504E0705DFEF7D5
:1036700095FE681C85B2BD42F8DB01200249086056
:10368000FFF79CFFBDE8F0819001214210B5FFF7E4
:103690000BFF0020FFF7E4FE962000F089FC6C226F
:1036A00000210748FFF7A4FF01226D210548FFF71D
:1036B0009FFF6C2200210448FFF71EFF10BD000091
:1036C0001C00002072050020F40500200FB4054BFB
:1036D00010B503A9044A029800F0DAF810BC5DF8AE
:1036E00014FB000051400008F005002002E008C86B
:1036F000121F08C1002AFAD170477047002001E06C
:1037000001C1121F002AFBD1704700002DE9FF5FA5
:1037100082B00021DDE90430020DDDF840B0034342
:1037200018D044F61050A2F2FF32424315141198FB
:1037300001281FD0A5EB0B00401C5FEA000A4FF0E8
:1037400000064E4FDFF83891B046504615D5CAF105
:10375000000413E0119801244AA3012801D16FEA63
:103760000B010298119AC0E90031C0E9024206B08B
:10377000BDE8F09FCBF10000DFE704460021404A9E
:10378000491842EB0450CDE9001012E0E00707D0E1
:1037900032463B4640464946FCF793FE8046894602
:1037A00032463B4610461946FCF78BFE06460F464E
:1037B0006410002CEAD1DDE90401DDE90023BAF14F
:1037C000000F06DAFCF77DFE42464B46FCF779FE19
:1037D00005E0FCF7E8FE42464B46FCF7E4FE0446F3
:1037E0000E460022284BFCF7A1FF03D84FF0FF3014
:1037F000014607E00022254B20463146FCF7BAFD82
:10380000FDF7E8F8102409E0002C0ADB0A22002367
:10381000FCF7EAFF039B30321A55641E50EA01029E
:10382000F2D1641C039AC4F111031444119A012AC1
:1038300003D0012208430DD10AE0084304D0002040
:103840004FF0110B119072E7A3EB0B056D1E0DE00D
:103850005B4504DD4FF0000205F1010504E003DAE9
:103860004FF00002A5F10105002AECD00298119951
:10387000C0E90231C0E9004579E7000000001440CA
:103880000000F03F300000000000F0430000E03F87
:103890002DE9FF4F95B09A46884606460025EEE191
:1038A000252877D100242746F94A0121039400E016
:1038B000044316F8013F203B01FA03F01042F7D110
:1038C00030782A2811D06FF02F033078A0F1300221
:1038D000092A16D8039A44F0020402EB820203EB91
:1038E00042021044761C0390EFE758F8042B039231
:1038F000002A03DA504244F40054039044F00204D6
:10390000761C30782E2816D116F8010F44F00404E6
:103910002A280DD06FF02F023078A0F13003092B48
:1039200009D807EB870302EB4303C718761CF3E7BC
:1039300058F8047B761C30786C280FD006DC4C28B5
:1039400017D068280DD06A2814D104E0742810D04C
:103950007A280FD10DE044F400140AE044F48014F6
:1039600001E044F440147278824202D104F58014DC
:10397000761C761C307866280BD013DC582877D05C
:1039800009DC002875D04528F6D04628F4D0472811
:103990001AD193E118E0632835D0642879D06528DE
:1039A00012D18BE1702873D008DC6728F1D0692828
:1039B0006FD06E280DD06F2806D1ACE073282CD0C4
:1039C000752874D0782853D05246179990476D1CAB
:1039D00054E1C4F30250022809D003280DD0D8F8CE
:1039E000001004280DD00D6008F1040846E1D8F855
:1039F0000010EA17C1E90052F6E7D8F800100D8070
:103A0000F2E70D70F0E718F8041B8DF800100020A5
:103A10008DF80100EB46012003E058F804BB4FF09D
:103A2000FF3061074FF0000102D40DE009F1010100
:103A30008946B9420FDA8145F8DB1BF809100029E5
:103A4000F4D108E009F1010189468142FADB1BF853
:103A500009100029F6D103985346A0EB0907214627
:103A60003846179A00F080FA284400EB090507E071
:103A700044E008E10DE01BF8010B5246179990470E
:103A8000B9F10109F7D2534621463846179AF2E0B8
:103A900039E00A21C4F302524FF0000B0091022AD0
:103AA00006D058F8040BC117032A09D00AE023E016
:103AB00008F1070020F00702F2E80201904605E055
:103AC00000B2C117042A01D140B2C117002906DA99
:103AD0000A460021404261EB02012D2202E022054C
:103AE00004D52B228DF80420012203E0E20701D047
:103AF0002022F7E7914657E00A2100E010214FF01D
:103B0000000B00910BE010214FF0000B44F0040477
:103B10000827009103E008204FF0000B0090C4F349
:103B20000252022A05D058F8040B0021032A08D0BB
:103B300008E008F1070020F00702F2E802019046D1
:103B400003E080B2042A00D1C0B24FF0000922077E
:103B50002AD53278702A07D0DDF800C08CF0100C1E
:103B60005CEA0B0C05D00EE040228DF80420012207
:103B700008E050EA010306D030238DF804308DF8B8
:103B8000052002229146009B83F0080353EA0B03B1
:103B90000AD150EA010201D1620705D530228DF821
:103BA00004204FF001097F1E3278582A04D039A230
:103BB0000C920CAA02920BE03BA2F9E75B46009A3A
:103BC000FCF712FE0C9B9B5C029A521E0292137031
:103BD00050EA0102F2D1029804A9081A00F1200B60
:103BE000600702D524F4803400E001275F4502DD40
:103BF000A7EB0B0000E0002000EB0B010090039806
:103C00004944401A0390E00306D453462146179ACC
:103C1000039800F0A9F90544002706E001A85246E0
:103C2000C05D179990476D1C7F1C4F45F6DBE00384
:103C30000CD553462146179A039800F095F9054490
:103C400004E030205246179990476D1C0099481E99
:103C500000900029F5DC08E00298029952460078AD
:103C6000491C0291179990476D1CBBF10001ABF103
:103C7000010BF1DC5BE100F065F90544761C30785E
:103C800000287FF40DAE19B02846BDE8F08F000083
:103C90000928010030313233343536373839616222
:103CA00063646566000000003031323334353637E6
:103CB000383941424344454600000000600700D4C3
:103CC000062708F1070020F00700F0E802238046ED
:103CD00003F0004C5FEA0C0001D097A009E020053A
:103CE00001D596A005E0E00701D095A001E0AFF274
:103CF0004C001390307823F0004365280CD006DC8C
:103D0000452809D046281DD047287FD13BE06628AA
:103D100018D067287AD136E00021112F01DB11205D
:103D200000E0781CCDE9000104A90CA8FFF7EEFC27
:103D3000DDE90D010C9A4FF0000B07F1010910921B
:103D400000914EE04FF000400097CDE9011004A92A
:103D50000CA8FFF7DBFCDDE90D020C9B0F994FF07F
:103D6000000B91461093009211B9791C00EB0109E8
:103D7000B7EB090003D4C0F1FF3B07F10109A9EB40
:103D80000700019042E0012F00DA01270021112FE6
:103D900001DD112000E03846CDE9000104A90CA89E
:103DA000FFF7B4FCDDE90D010C9A00914FF0000B18
:103DB000B946109221070FD4009A4A4503DA91467A
:103DC00001E0A9F10109B9F1010F05DD109AA9F18E
:103DD0000101515C3029F4D0B84202DA10F1040F2D
:103DE00003DA0121CDE9011010E0002803DC83444F
:103DF000A9EB000102E0411C494500DD8946A0EB2A
:103E00000B00401C01904FF000400290200705D4A9
:103E10000198484502DB4FF0FF30019000208DF8FB
:103E20004B0002980DF14B07B0F1004F25D0022056
:103E30000C902B200D90029800280CDA4042029042
:103E40002D200D9007E00A210298FCF7B7FC3031D5
:103E5000029007F8011D0C99481E0C900029F2DC15
:103E600002980028EFD1791E0D980870307800F084
:103E7000200040F0450007F8020D11A8C01BC01D2E
:103E800002901398007800B1012000EB090101981D
:103E900001EBE071029801440398401A401E039020
:103EA000E00306D453462146179A039800F05CF8C5
:103EB00005441398007818B15246179990476D1C25
:103EC000E00323D553462146179A039800F04CF897
:103ED00005441BE0BBF1000F07DB0098584504DDEB
:103EE0001098179910F80B0001E0179930205246EE
:103EF000904701980BF1010B401E05F1010501905F
:103F000004D12E205246179990476D1CB9F100013B
:103F1000A9F10109DEDC05E017F8010B52461799FB
:103F200090476D1C0299481E02900029F4DC53460C
:103F30002146179A03989EE62D0000002B000000F2
:103F4000200000002DE9F041044600251E461746DA
:103F5000880404D405E039462020B0476D1C641E57
:103F6000F9D52846BDE8F0812DE9F0410446002549
:103F70001E469046C80301D5302700E0202788045C
:103F800004D505E041463846B0476D1C641EF9D59E
:103F90002846BDE8F08170B504460025104603E0D0
:103FA0000E5C66556D1C401C9842F9DB70BD00002C
:103FB00070B5044602F018F8012810D00B480088AC
:103FC000844206D309480088B4FBF0F5284601F086
:103FD0008FF906480088B4FBF0F100FB11444FF460
:103FE0007A7104FB01F000F003F870BDD6000020E8
:103FF00070B5034600224FF0E02675690D4E367805
:1040000003FB06F44FF0E026B16910E04FF0E02624
:10401000B06988420BD0884202D20E1A324402E0C4
:104020002E1A0E4432440146A24200D300E0EDE7CE
:1040300000BF70BDD400002030B50446002504E068
:104040004FF47A70FFF7D4FF6D1CA542F8D330BD52
:1040500070B504460D46012008490860E1B20848E1
:10406000FFF7F7F900BF80210548FFF725F9002881
:10407000F9D0002001490860204670BDA48121428A
:104080000044004002460B46002104E0505C08B1A9
:1040900000207047491C9942F8DB0120F9E770B510
:1040A00005460C4645F25550FDF75CF82846FDF7ED
:1040B0004DF82046FDF750F8FDF740F8FDF732F8CF
:1040C00070BD00001FB54FF44070FDF7A9F84820FF
:1040D000FEF7F2FC4FF41660FFF77EF8FDF762F989
:1040E00040F2671140F28F10FEF7CEFF4FF496506A
:1040F000FDF782FBFCF7AAFEFDF732FFFEF74EFD4F
:10410000FEF7CAF81F482049204A214BCDE900326A
:10411000CDE902101F4B204A20492148FCF7ECFC56
:1041200040F2CF2140F2F310FDF74EF940F2CF21DB
:1041300040F2F310FDF79AF940F2CF2140F2F3106C
:10414000FDF7E6F941F61F4142F20F70FEF77AFDE6
:104150004FF47A510520FFF7A2FF0220FCF79EFEE4
:10416000AA211048FEF739FF0020FDF717FA0020BA
:10417000FDF71EFA0020FDF723FA00F015F800BF46
:10418000FEE70000900500208E0500208C05002031
:104190008A05002088050020930500209205002054
:1041A00087050020000400401CB5064800210B468E
:1041B0008022CDE9001004A1064801F0E5FE01F0DF
:1041C00033FA1CBD6405002073746172745F7461FE
:1041D000736B0000594E00082DE9F04105460E466C
:1041E0001C4807681C480068001D00F0C3FE50B959
:1041F0001948006890F82C10012088401749096878
:10420000814316480160681C38B936B1124801680C
:10421000091D134800F0ECFE1AE07C190E480068F6
:104220004460BC4207D20C480168091D0D48006873
:1042300000F0C4FE0CE008480168091D0A48006847
:1042400000F0BCFE09480068844201D207480460BF
:10425000BDE8F08104010020F000002008010020EA
:10426000800B0020F8000020F40000202001002036
:1042700010B5044600F0C8FE23480068401C2249DF
:1042800008602248006840B9204804600846006879
:1042900001280DD100F0E4F90AE01D48006838B9A2
:1042A0001A480068C06AE16A884201D81748046069
:1042B00018480068401C1749086094F82C10012029
:1042C000884015490968084313490860E16A01EB11
:1042D0008101124A02EB8100211D00F089FE00F0ED
:1042E000D7FE0B48006868B108480068C06AE16AF8
:1042F000884207D24FF0805009490860BFF34F8FC2
:10430000BFF36F8F10BD000000010020F0000020FF
:104310000C0100201C01002008010020B008002032
:1043200004ED00E010B500F06FFE10480068D0B951
:104330000F4800F033FE0F4800F030FE0C480E49E5
:1043400008600C480D49086000220C210A2001F089
:1043500087FA064908600846006820B108A10348AA
:10436000006800F089FF00F093FE10BD34010020CA
:10437000940B0020A80B00202C010020300100200D
:10438000546D72510000000070B523E001F0A2F9F5
:104390001348006808B9012000E00020054601F03C
:1043A000AFFFBDB900F030FE0D48C068C468201DE5
:1043B00000F0E0FD0B480068401E0A4908600A480A
:1043C0000068401E0849086000F062FE204600F0C8
:1043D00060F800BF044800680028D7D170BD000015
:1043E0006C0B002000010020FC00002070B504468A
:1043F0000D46206C70B1216CE0680844E060616893
:10440000E068884201D32068E0602846226CE168B9
:10441000FBF7D6FE70BD2DE9F04104460F46154668
:104420004FF00008A66B206C40B9206860BB606844
:1044300001F0A0FE80460020606025E07DB939468D
:10444000226CA068FBF7BCFE216CA0680844A06049
:10445000D4E90110884217D32068A06014E03946DF
:10446000226CE068FBF7ACFE216CE068401AE0606B
:104470002168E068884203D2216C6068401AE060DD
:10448000022D01D106B1761E701CA0634046BDE826
:10449000F08110B50446206B00F032FE204600F09B
:1044A0002FFE10BD0146084A126812680AB901229F
:1044B00000E000220A600A6822B9034A1268D26842
:1044C000106800E0002070472C01002030B54FF448
:1044D0002053174800F007042CB1C01D20F007003E
:1044E000134C041B1B1B0246124C22600024114D6E
:1044F0006C60D018083820F007000F4C20600024B2
:104500000D4D2D686C600C4D2D682C601146441AC1
:104510004C60094C24680C60084D4C682C60084DB8
:104520004C682C604FF00044064D2C6030BD0000FC
:104530000C0C00204C010020540100205C010020E4
:10454000580100206001002000BFFFF71DFF064852
:1045500000680128F9D94FF0805004490860BFF382
:104560004F8FBFF36F8FF0E7B008002004ED00E03D
:104570002DE9F04106460D4617469846069C0DB9B2
:10458000246000E02760E66325640121204601F0F5
:10459000ADFA0020A064BDE8F08100002DE9FF5FC6
:1045A00081460F469246DDE90E6B109CAAF1010090
:1045B000216B01EB800828F0070808F0070008B914
:1045C000012000E0002028B940F22B321BA120A0DE
:1045D000FFF77CF8002507E0795D04F134004155D0
:1045E000785D00B902E06D1C102DF5D300BF0021ED
:1045F00043200155202E00D31F26E662666400206A
:10460000A064201D00F0D7FC04F1180000F0D3FCDA
:104610002461C6F12000A06164620020E06484F897
:10462000500049464046039A00F004FC2060BBF16C
:10463000000F01D0CBF80040BDE8FF9F2E2E5C4656
:1046400072656552544F535C7461736B732E6300D3
:104650004572726F723A25732C25640D0A000000B2
:1046600010B5002407E004EB84010F4A02EB81003F
:1046700000F094FC641C202CF5D30C4800F08EFC58
:104680000B4800F08BFC0B4800F088FC0A4800F057
:1046900085FC0A4800F082FC044809490860044887
:1046A0000849086010BD0000B0080020300B002051
:1046B000440B0020580B00206C0B0020800B0020C6
:1046C000F4000020F800002010B50146164800E074
:1046D000006803688B42FBD30246436813448B4255
:1046E00004D143684C682344436001460A464B6842
:1046F00013440468A34211D10C4C03682468A342FC
:1047000008D04B680468646823444B6003681B68E6
:104710000B6005E0054B1B680B6001E003680B6054
:10472000884200D0016010BD4C01002054010020DF
:104730002DE9F04104460D4616461F464FF000088D
:1047400065602461B5420CD8F01BA169884202D390
:104750004FF0010811E0211D0948006800F02EFC0F
:104760000BE0BE4204D2BD4202D34FF0010804E088
:10477000211D0448006800F021FC4046BDE8F0819E
:10478000300100202C01002070B5054600F03CFCF3
:10479000A86B08B9012400E0002400F079FC204651
:1047A00070BD70B5054600F02FFCA86BE96B884220
:1047B00001D1012400E0002400F06AFC204670BD15
:1047C0002DE9F3410D460098846C00272CB940F682
:1047D000CE121AA128A0FEF779FFA06BE16B8842E8
:1047E00001D2012000E0002028B940F6CF1213A129
:1047F00021A0FEF76BFFA06BE16B88421BD294F9FE
:1048000045602A4669462046FFF705FE0746701CAC
:1048100060B9606A08B9012000E0002050B904F1D5
:10482000240001F013FD28B1012703E0701C40B201
:1048300084F8450000BF3846BDE8FC812E2E5C2E72
:104840002E5C2E2E5C73746D33322D636F6E74721A
:104850006F6C205F6C69616E77616E675C636F6E11
:1048600074726F6C5C4672656552544F535C71751F
:104870006575652E630000004572726F723A25738C
:104880002C25640D0A000000F8B505460F461348B4
:104890000068C068C468201D00F06CFBE069012856
:1048A00018D1A06941192B463A462046FFF740FF30
:1048B00080B1002003462A4601460090204601F0C0
:1048C000E9FD06462EB94FF4027205A10AA0FEF7D3
:1048D000FDFE00BF2046616A8847F8BD2C0100201C
:1048E0002E2E5C4672656552544F535C74696D653B
:1048F00072732E63000000004572726F723A257366
:104900002C25640D0A00000070B586B060E00398A5
:1049100000285DDB059C606908B9012000E00020EB
:1049200010B9201D00F026FB02A800F0C7F80546CC
:1049300003980A284AD2DFE800F00905072C2E4523
:1049400006082D2F00BF00BF00BF00BF0498A2695A
:10495000811803462A462046FFF7EAFEC0B12046EA
:10496000616A8847E069012812D10020009004980C
:10497000A169421800231946204601F08BFD064626
:104980002EB940F2213218A11DA0FEF79FFE00BFF4
:104990001DE000BF1BE000BF0498A061A06908B142
:1049A000012000E0002028B94FF44E720EA114A09F
:1049B000FEF78CFEA06941192B462A462046FFF7D8
:1049C000B7FE04E0204600F09BFB00E000BF00BF04
:1049D00000231A4603A90E48006800F08FFF002844
:1049E00095D106B070BD00002E2E5C4672656552F2
:1049F000544F535C74696D6572732E630000000040
:104A00004572726F723A25732C25640D0A000000FE
:104A100034010020F8B505460C4600F05BFE684600
:104A200000F04CF80646009820BB44B9B54206D8C1
:104A300001F066FC31462846FFF726FF1CE03CB13A
:104A40000E480068006808B9012000E00020044614
:104A5000A91B22460A48006800F024FC01F050FC23
:104A600050B94FF0805007490860BFF34F8FBFF334
:104A70006F8F01E001F044FCF8BD00003001002020
:104A80003401002004ED00E00A490968096809B909
:104A9000012100E0002121B14FF0FF31064A1160F1
:104AA00006E004490968C968C868034A416811609A
:104AB00070470000F40000202001002070B504467B
:104AC00001F0A2FA054607480068854204D200F0CA
:104AD0000BF80120206001E0002020600148056003
:104AE000284670BD3C0100202DE9F8432DE0214807
:104AF0000068C06805681F480068C068C468201D59
:104B000000F038FA2046616A8847E06901281CD124
:104B1000A0694619AE4207D966602461211D154877
:104B2000006800F04BFA10E0002003462A460146D8
:104B30000090204601F0AEFC07462FB940F29232B9
:104B40000DA113A0FEF7C2FD00BF0A48006800686F
:104B500008B9012000E000200028C8D00548D0F89E
:104B600000800F480068034908600D48C0F80080C5
:104B7000BDE8F8832C0100202E2E5C46726565523C
:104B8000544F535C74696D6572732E6300000000AE
:104B90004572726F723A25732C25640D0A0000006D
:104BA000300100200B480068401C08B9012000E0DB
:104BB000002020B9F42208A112A0FEF787FD00BF53
:104BC000502080F31188BFF34F8FBFF36F8F00BF6A
:104BD00000BFFEE7400100202E2E5C467265655244
:104BE000544F535C706F727461626C655C525644D2
:104BF000535C41524D5F434D335C706F72742E6352
:104C0000000000004572726F723A25732C25640D06
:104C10000A00000008B500BF6846FFF743FC0446E1
:104C200020460099FFF7F6FEFFF76EFEF4E770B539
:104C3000044600F0E9F994F945501AE0A06C38B147
:104C400000212046FFF7BCFD88B100F011FC0EE00A
:104C5000606A08B9012000E0002038B904F124009E
:104C600001F0F4FA18B100F003FC00E003E0681E64
:104C700045B2002DE2DC00BFFF2084F8450000F0C3
:104C800007FA00F0C1F994F9445010E0206908B91E
:104C9000012000E0002048B904F1100001F0D6FA2C
:104CA00008B100F0E5FB681E45B200E001E0002D10
:104CB000ECDC00BFFF2084F8440000F0E9F970BD8F
:104CC0002DE9F04104464FF0000800F003FD3E4896
:104CD000006808B9FFF7FAFB3C480068204000284C
:104CE0005FD1A4B1083404F0070080B104F00700DC
:104CF000C0F10800044404F0070008B9012000E0F6
:104D0000002020B9BF2232A13BA0FEF7DFFC002C1F
:104D100047D03D480068844243D83C4E3046056841
:104D200001E02E462D686868A04202D2286800285B
:104D3000F7D125480068854233D0306800F1080873
:104D4000286830606868001B102813D92F1907F0F5
:104D5000070008B9012000E0002020B9EC221CA1C6
:104D600025A0FEF7B3FC6868001B78606C603846CD
:104D7000FFF7AAFC244968680968081A22490860F4
:104D80000846006822490968884203D21E48006824
:104D90001F4908600D496868096808436860002079
:104DA000286001F0ADFA08F0070008B9012000E022
:104DB000002028B94FF4967205A10FA0FEF786FCDB
:104DC0004046BDE8F0810000540100206001002051
:104DD0002E2E5C4672656552544F535C706F727430
:104DE00061626C655C4D656D4D616E675C686561A7
:104DF000705F342E630000004572726F723A257343
:104E00002C25640D0A000000580100204C010020F0
:104E10005C0100200648006830B10549096801F1CD
:104E20004800896C491C0160014800687047000017
:104E3000F0000020001F4FF080730360001F21F07E
:104E400001030360001F034B036014380260203825
:104E500070470000A54B00081CB5044600F0D4F8CC
:104E60000948012100234A02CDE9001007A10E489C
:104E700001F08AF80D4908600D48006800F072FAE8
:104E800000F006F91CBD00006805002053656E7334
:104E90006F725F436F6D6D756E69636174696F6E7C
:104EA0005F7461736B0000008D240008C005002052
:104EB000640500201CB528492848FCF73FFF274817
:104EC0000078C0EB00102449097801EB80002449E8
:104ED00008802448007800EBC00040000E382249CA
:104EE000095C2048007800EBC00040000F381E4AE3
:104EF000105CC0EB001001EB80001C4908801848D2
:104F000000880988884220DB0020009003460122A7
:104F10000921019040F2E770FDF734F9114800785B
:104F2000062806D1012012490870FEF7AFFB0120C8
:104F30001CBD0C480078401C0D490870FEF7A6FB0C
:104F400008480078401CC0B2F2E7064800780849DB
:104F5000087004480078EBE77F0500207E050020FC
:104F600018000020870500201C0000201A000020E7
:104F70007205002001460A69D1E901309860D1E943
:104F8000010358605068884201D188685060002051
:104F900008611068401E10601068704700F1080139
:104FA00041604FF0FF31816000F10801C160016193
:104FB00000210160704700210161704710B5024671
:104FC0000B685C1C0CB9106907E002F1080000E0F6
:104FD0004068446824689C42FAD944684C604C6834
:104FE000A160886041600A611468641C146010BD8F
:104FF00042684A6093688B60936859609160086169
:1050000003685B1C0360704710B500BF502080F33D
:105010001188BFF34F8FBFF36F8F00BF0B4800683D
:10502000401C0A4908600846006801280DD108485C
:105030000068C0B208B9012000E0002028B94FF490
:10504000BD7204A10EA0FEF741FB10BD400100207F
:1050500004ED00E02E2E5C4672656552544F535CA1
:10506000706F727461626C655C525644535C41525D
:105070004D5F434D335C706F72742E63000000000F
:105080004572726F723A25732C25640D0A00000078
:1050900010B50B48006828B940F2811209A114A08C
:1050A000FEF714FB06480068401E054908600846E4
:1050B000006820B9002080F3118800BF00BF10BD38
:1050C000400100202E2E5C4672656552544F535CA1
:1050D000706F727461626C655C525644535C4152ED
:1050E0004D5F434D335C706F72742E63000000009F
:1050F0004572726F723A25732C25640D0A00000008
:1051000070B506463546002E35D0083D2C461A4966
:1051100060680968084008B1012000E0002028B953
:105120004FF4A07215A11FA0FEF7D0FA206808B9AD
:10513000012000E0002028B940F241120FA119A07F
:10514000FEF7C4FA0C4960680968084098B1206805
:1051500088B90949606809688843606000F0BAFA54
:105160001449606809680844124908602046FFF73E
:10517000ABFA01F0C5F870BD600100202E2E5C4630
:1051800072656552544F535C706F727461626C65E6
:105190005C4D656D4D616E675C686561705F342E56
:1051A000630000004572726F723A25732C25640DFE
:1051B0000A00000058010020064800684FF47A7188
:1051C000B0FBF1F0401E4FF0E0214861072008617C
:1051D000704700000000002070B5FAF7DBFF0546BD
:1051E000102D11D305F1E02090F8F043104800781D
:1051F000844201DB012000E0002028B94FF42A722C
:105200000CA117A0FEF762FA1948006800F4E060EC
:1052100018490968884201D8012000E0002028B917
:105220004FF42E7203A10EA0FEF750FA70BD0000DD
:10523000440100202E2E5C4672656552544F535C2B
:10524000706F727461626C655C525644535C41527B
:105250004D5F434D335C706F72742E63000000002D
:105260004572726F723A25732C25640D0A00000096
:105270000CED00E048010020024600200BE0084B46
:1052800053F8303033B9064B43F8301003EBC0030A
:105290005A6002E0401C0A28F1D300BF70470000AA
:1052A000BC0B00202DE9F04105460E4617462C4662
:1052B000FFF7AAFE94F94400401C10B9002084F8BE
:1052C000440094F94500401C10B9002084F84500C2
:1052D000FFF7DEFEA06B28B93A46314604F1240000
:1052E00000F0F6F82046FFF7A2FCBDE8F0810000D0
:1052F00070B504460025ACB10F48006808B901201C
:1053000000E0002028B940F2CF420CA110A0FEF727
:10531000DDF900F0DFF900212046FEF75DFF00F027
:10532000EFFF05463DB94FF080500D490860BFF3CF
:105330004F8FBFF36F8F70BD280100202E2E5C466B
:1053400072656552544F535C7461736B732E6300C6
:105350004572726F723A25732C25640D0A000000A5
:1053600004ED00E070B50546FFF74EFE15B92D4877
:10537000006800E028460446201DFFF7FBFD78B9D1
:10538000E06A00EB8000284951F8200040B994F809
:105390002C10012088402549096881432348016079
:1053A000A06A18B104F11800FFF7E4FD2048006876
:1053B000401C1F4908601B480068844209D1211D18
:1053C0001C48FFF715FE1C480068401C1A4908607D
:1053D00009E01A480068401E184908602046FFF797
:1053E00058F8FFF751FBFFF753FE15480068C0B1AE
:1053F0000C480068844214D11248006808B90120A2
:1054000000E0002028B940F265420FA113A0FEF78A
:105410005DF94FF0805015490860BFF34F8FBFF31F
:105420006F8F70BDF0000020B00800200801002040
:105430001C0100206C0B0020FC000020000100205B
:105440000C010020280100202E2E5C46726565525A
:10545000544F535C7461736B732E63004572726FAB
:10546000723A25732C25640D0A00000004ED00E05B
:1054700001200149086070471401002070B50446FE
:105480000D462CB940F6063207A10CA0FEF71EF916
:105490000E48016818312046FFF790FD012128468B
:1054A000FEF79AFE70BD00002E2E5C4672656552B6
:1054B000544F535C7461736B732E63004572726F4B
:1054C000723A25732C25640D0A000000F0000020BC
:1054D00070B505460E4614462DB940F6313209A185
:1054E0000DA0FEF7F3F81048016818312846FFF7C1
:1054F0007FFD0CB14FF0FF3621463046FEF76CFEC3
:1055000070BD00002E2E5C4672656552544F535C90
:105510007461736B732E63004572726F723A2573F8
:105520002C25640D0A000000F000002070B505462F
:105530002C46002D4BD02649E06A0968C96A88428A
:1055400045D2A06900F0004028B921480068C06A2F
:10555000C0F12000A061E16A01EB81011D4A02EB6C
:1055600081016069884201D1012000E0002050B330
:10557000201DFFF7FFFC78B9E06A00EB80001549B9
:1055800051F8200040B994F82C10012088401249AD
:1055900009688143104801600D480068C06AE062F4
:1055A00094F82C10012088400B49096808430A49E7
:1055B0000860E16A01EB8101064A02EB8100211DCE
:1055C000FFF716FD03E002480068C06AE06270BDA4
:1055D000F0000020B00800200801002010B50446AB
:1055E0002CB940F6C13205A109A0FEF76FF80C48AE
:1055F000006820600B480068606010BD2E2E5C467D
:1056000072656552544F535C7461736B732E630003
:105610004572726F723A25732C25640D0A000000E2
:1056200018010020040100201CB51A4800210B4677
:105630008022CDE9001018A1194800F0A5FC04460D
:10564000012C02D100F0ECFE0446012C15D100BF64
:10565000502080F31188BFF34F8FBFF36F8F00BFCF
:105660004FF0FF300F49086001200F49086000200B
:105670000E49086000F08AF80BE0601C08B10120B8
:1056800000E0002028B940F2847209A10DA0FEF7C5
:105690001DF81CBD2401002049444C4500000000B9
:1056A00049450008200100200C01002004010020D1
:1056B0002E2E5C4672656552544F535C7461736B59
:1056C000732E63004572726F723A25732C25640D38
:1056D0000A00000002480068401C01490860704749
:1056E0002801002010B51B48006818B101201A4994
:1056F00008602DE000201849086018480068B0FADA
:1057000080F0C0F11F0404EB8400154951F820001B
:1057100008B1012000E0002028B940F6F62211A1CE
:1057200015A0FDF7D3FF04EB84010D4A02EB8100C5
:1057300041684968416000F1080142688A4202D12B
:105740004168496841604168C9680F4A116000BFFB
:1057500010BD0000280100201401002008010020D5
:10576000B00800202E2E5C4672656552544F535C83
:105770007461736B732E63004572726F723A257396
:105780002C25640D0A000000F00000201CB5224802
:10579000014609780191FF210246117001460978FE
:1057A00000919DF8001001F050011C4A1170072172
:1057B0001B4A116009E01A490968491E184A11601C
:1057C0009DF800104906090E00919DF8001001F0A7
:1057D00080018029EFD0124909680902104A11603E
:1057E0001146098801F4E06111600B4A01991170BA
:1057F0000C48006840F470000A49086008460068D8
:1058000040F070400860FFF7D7FC002006490860B0
:10581000FAF78AFC00201CBD00E400E044010020EF
:105820004801002020ED00E04001002010B500BF3D
:10583000502080F31188BFF34F8FBFF36F8F00BFED
:1058400000F0E8FB18B14FF080500449086000BF39
:10585000002080F3118800BF10BD000004ED00E0BF
:105860002DE9F84305460E4690460DB1012000E0B3
:10587000002028B94FF4C4720DA11CA0FDF726FF2B
:105880000EB9002701E005FB06F707F14C00FFF712
:1058900017FA044644B104F14C0943464A463146DE
:1058A00028460094FEF764FE2046BDE8F883000019
:1058B0002E2E5C2E2E5C2E2E5C73746D33322D6377
:1058C0006F6E74726F6C205F6C69616E77616E676A
:1058D0005C636F6E74726F6C5C4672656552544F98
:1058E000535C71756575652E630000004572726FBB
:1058F000723A25732C25640D0A0000002DE9FF473C
:1059000082B005460E461F464FF0000A2C462CB9C1
:1059100040F2DC4261A170A0FDF7D8FE0EB9206C08
:1059200008B9012000E0002028B940F2DD425BA167
:1059300069A0FDF7CBFE00F057FB08B9049808B941
:10594000012000E0002028B94FF49C6253A162A01E
:10595000FDF7BCFE00BFFFF757FBD4F83890B9F154
:10596000000F3DD0D4F80C8031462046FEF73EFDB6
:10597000DFB9A9F10100A063206810B9FFF74AFA66
:105980006060206908B9012000E0002010BB04F12C
:10599000100000F05BFCE8B14FF080505249086005
:1059A000BFF34F8FBFF36F8F14E0C4F80C80606AB1
:1059B00008B9012000E0002060B904F1240000F0E3
:1059C00045FC38B14FF0805047490860BFF34F8F16
:1059D000BFF36F8FFFF75CFB012006B0BDE8F087D7
:1059E000049818B9FFF754FB0020F6E7BAF1000F4E
:1059F00004D16846FFF7F2FD4FF0010AFFF748FBBC
:105A0000FFF768FEFFF700FB94F94400401C10B953
:105A1000002084F8440094F94500401C10B900208F
:105A200084F84500FFF734FB04A9684600F05CFAEF
:105A300040BB2046FEF7A8FEF0B1206830B9FFF762
:105A4000E3FA6068FFF772FDFFF722FB04F1240020
:105A50000499FFF713FD2046FFF7E9F800F050FC2A
:105A600000287FF478AF4FF080501F490860BFF3E3
:105A70004F8FBFF36F8F6EE72046FFF7D8F800F027
:105A80003FFC68E72046FFF7D2F800F039FC2046DB
:105A9000FEF77AFE0028EED000209EE72E2E5C2E28
:105AA0002E5C2E2E5C73746D33322D636F6E7472A8
:105AB0006F6C205F6C69616E77616E675C636F6E9F
:105AC00074726F6C5C4672656552544F535C7175AD
:105AD0006575652E630000004572726F723A25731A
:105AE0002C25640D0A00000004ED00E070B50546A9
:105AF0000E462C462CB940F21B121EA12CA0FDF71D
:105B0000E5FDFFF781FAD4E90F12206801FB0200DE
:105B100060600020A0632068A060E06B401E226CE3
:105B2000216800FB0210E060FF2084F8440084F844
:105B300045009EB9206908B9012000E00020A8B9FD
:105B400004F1100000F082FB80B14FF080501C493E
:105B50000860BFF34F8FBFF36F8F07E004F11000B1
:105B6000FFF71CFA04F12400FFF718FAFFF790FA88
:105B7000012070BD2E2E5C2E2E5C2E2E5C73746D5B
:105B800033322D636F6E74726F6C205F6C69616E5F
:105B900077616E675C636F6E74726F6C5C46726582
:105BA0006552544F535C71756575652E6300000036
:105BB0004572726F723A25732C25640D0A0000003D
:105BC00004ED00E02DE9FF4383B0064688461D46FC
:105BD0004FF0000934462CB940F2D92260A16FA0E1
:105BE000FDF774FDB8F1000F01D1206C08B9012058
:105BF00000E0002028B940F2DA2259A167A0FDF7A1
:105C000065FD022D02D1E06B012801D1012000E0E9
:105C1000002028B940F2DB2251A160A0FDF756FD1B
:105C200000F0E2F908B9059808B9012000E0002069
:105C300028B940F2DE224AA158A0FDF747FD00BF77
:105C4000FFF7E2F9A06BE16B884201D3022D38D156
:105C50002A4641462046FEF7DEFB0746A06C68B1A7
:105C600029462046FEF7ACFD28B34FF080504F493F
:105C70000860BFF34F8FBFF36F8F1CE0606A08B9F5
:105C8000012000E0002068B904F1240000F0DEFAF1
:105C900088B14FF0805045490860BFF34F8FBFF384
:105CA0006F8F08E03FB14FF0805040490860BFF36C
:105CB0004F8FBFF36F8FFFF7EBF9012007B0BDE8FF
:105CC000F083059818B9FFF7E3F90020F6E7B9F17A
:105CD000000F04D101A8FFF781FC4FF00109FFF785
:105CE000D7F9FFF7F7FCFFF78FF994F94400401C50
:105CF00010B9002084F8440094F94500401C10B904
:105D0000002084F84500FFF7C3F905A901A800F0B9
:105D1000EBF8F0B92046FEF744FDA0B104F1100005
:105D20000599FFF7ABFB2046FEF781FF00F0E8FA8C
:105D3000002885D14FF080501C490860BFF34F8F79
:105D4000BFF36F8F7CE72046FEF771FF00F0D8FAB3
:105D500076E72046FEF76BFF00F0D2FA0020ADE7B1
:105D60002E2E5C2E2E5C2E2E5C73746D33322D63C2
:105D70006F6E74726F6C205F6C69616E77616E67B5
:105D80005C636F6E74726F6C5C4672656552544FE3
:105D9000535C71756575652E630000004572726F06
:105DA000723A25732C25640D0A00000004ED00E012
:105DB0002DE9F05F80468A4615461E4644462CB9BA
:105DC00040F29F3235A144A0FDF780FCBAF1000FEC
:105DD00001D1206C08B9012000E0002028B94FF45F
:105DE00068722EA13CA0FDF771FC022E02D1E06B7F
:105DF000012801D1012000E0002028B940F2A132A1
:105E000026A135A0FDF762FCFFF7E6F900BF50219F
:105E1000EFF3118081F31188BFF34F8FBFF36F8FC2
:105E200000BF0746A06BE16B884201D3022E2BD145
:105E300094F945B0324651462046FEF7ECFA0BF194
:105E40000100C8B9A06C40B131462046FEF7B8FC4D
:105E5000B8B1B5B10120286013E0606A08B901202B
:105E600000E0002068B904F1240000F0EFF940B12F
:105E70003DB10120286004E00BF1010040B284F83C
:105E800045004FF0010901E04FF0000900BF87F322
:105E9000118800BF4846BDE8F09F00002E2E5C2E02
:105EA0002E5C2E2E5C73746D33322D636F6E7472A4
:105EB0006F6C205F6C69616E77616E675C636F6E9B
:105EC00074726F6C5C4672656552544F535C7175A9
:105ED0006575652E630000004572726F723A257316
:105EE0002C25640D0A0000002DE9F04104460D4602
:105EF0002CB940F6CB3219A11DA0FDF7E7FB2DB957
:105F000040F6CC3215A11AA0FDF7E0FBFFF77CF8B4
:105F10001B4807682868401C08B9002619E0194981
:105F200020680968884204D06068B84201D8012618
:105F30000FE06068381A2968884209D228686168C9
:105F4000791A401A28602046FFF748FB002600E037
:105F50000126FFF79DF83046BDE8F0812E2E5C4605
:105F600072656552544F535C7461736B732E63009A
:105F70004572726F723A25732C25640D0A00000079
:105F800004010020180100202DE9FF4F85B0804654
:105F900089461746DDE912ABB800FEF791FE0646CA
:105FA00056B15420FEF78CFE04460CB1266304E083
:105FB0003046FFF7A5F800E000247CB10020CDE9D1
:105FC00000ABCDE902403A4649464046089BFEF701
:105FD000E5FA2046FEF74CF9012501E04FF0FF35C8
:105FE000284609B0BDE8F08F0549096809B90120C4
:105FF00005E00449096809B9022000E00020704763
:106000000C010020280100200149086870470000A9
:10601000040100202DE9F0414FF0000841480068DC
:10602000002872D140480068451C3F480560EDB922
:106030003E480068006808B9012000E0002028B947
:1060400040F6D9123AA13FA0FDF740FB3748076858
:1060500040480068354908603E4807603E4800688F
:10606000401C3D490860FEF70FFD00BF3B4800683B
:1060700085423CD300BF2D480068006808B9012064
:1060800000E0002020B14FF0FF30344908602DE0DF
:1060900026480068C068C4686668B54202D22F48C6
:1060A000066023E0201DFEF765FFA06A18B104F129
:1060B0001800FEF75FFF94F82C1001208840284953
:1060C0000968084326490860E16A01EB8101254A15
:1060D00002EB8100211DFEF78BFF2349E06A09686E
:1060E000C96A8842C7D34FF00108C4E700BF1E4801
:1060F0000068C06A00EB80001A4951F820000128AE
:1061000001D94FF0010805E0FFE718480068401C7E
:10611000164908601648006808B14FF0010840466B
:10612000BDE8F0812801002004010020F4000020D7
:106130002E2E5C4672656552544F535C7461736BCE
:10614000732E63004572726F723A25732C25640DAD
:106150000A000000F80000201801002020010020A3
:1061600008010020B0080020F000002010010020ED
:106170001401002070B505462C460026002D4BD09A
:1061800026480068844201D1012000E0002028B99F
:1061900040F6C76222A127A0FDF798FAA06C28B9A3
:1061A00040F6C9621EA123A0FDF790FAA06C401E24
:1061B000A064616CE06A88422ED0A06C60BB201D98
:1061C000FEF7D8FE78B9E06A00EB80001D4951F86F
:1061D000200040B994F82C10012088401A49096821
:1061E000814319480160606CE062E06AC0F1200000
:1061F000A06194F82C1001208840134909680843D5
:1062000011490860E16A01EB81010E4A02EB81004D
:10621000211DFEF7EDFE0126304670BDF000002086
:106220002E2E5C4672656552544F535C7461736BDD
:10623000732E63004572726F723A25732C25640DBC
:106240000A000000B00800200801002070B50646D2
:10625000F068C4682CB940F661321AA11EA0FDF79F
:1062600035FA04F11800FEF785FE1F480068A8B94A
:10627000201DFEF77FFE94F82C10012088401B495A
:106280000968084319490860E16A01EB8101184A6D
:1062900002EB8100211DFEF7ABFE04E004F11801C2
:1062A0001448FEF7A5FE1449E06A0968C96A8842E5
:1062B00004D9012501201149086000E00025284685
:1062C00070BD00002E2E5C4672656552544F535CC3
:1062D0007461736B732E63004572726F723A25732B
:1062E0002C25640D0A000000280100200801002070
:1062F000B0080020580B0020F000002014010020FE
:1063000070B5002400263448006828B94FF4FD62B7
:1063100032A137A0FDF7DAF9FEF776FE2E480068C5
:10632000401E2D4908600846006800284FD13448B7
:10633000006800284BD024E03248C068C46804F1EB
:106340001800FEF717FE201DFEF714FE94F82C101F
:10635000012088402C49096808432B490860E16AFC
:1063600001EB8101294A02EB8100211DFEF740FE6D
:106370002749E06A0968C96A884202D30120254991
:1063800008602048006808B9012000E000200028CB
:10639000D2D00CB1FEF778FB1F48056865B100BF8D
:1063A000FFF738FE10B101201A4908606D1E002D5C
:1063B000F6D10020184908601648006838B1012657
:1063C000300716490860BFF34F8FBFF36F8FFEF79A
:1063D0005FFE304670BD0000280100202E2E5C4676
:1063E00072656552544F535C7461736B732E630016
:1063F0004572726F723A25732C25640D0A000000F5
:1064000000010020580B002008010020B0080020E7
:10641000F0000020140100201001002004ED00E035
:106420001CB50024FDF77EFF0B48006858B10B48EF
:106430001F2100234FF48072CDE9001008A10A4803
:10644000FFF7A2FD04462CB940F2331207A10DA0BC
:10645000FDF73CF920461CBD340100203801002026
:10646000546D722053766300154C00082E2E5C4646
:1064700072656552544F535C74696D6572732E6317
:10648000000000004572726F723A25732C25640D6E
:106490000A0000002DE9FE4304460D4616461F463D
:1064A000DDF828804FF000092CB94FF4D37216A103
:1064B0001BA0FDF70BF91E48006810B3009501966C
:1064C0000294062D15DAFFF78FFD022808D100236C
:1064D0004246694616480068FFF774FB814610E0A3
:1064E00000231A46694612480068FFF76BFB814695
:1064F00007E000233A4669460D480068FFF758FC5C
:1065000081464846BDE8FE832E2E5C467265655284
:10651000544F535C74696D6572732E630000000004
:106520004572726F723A25732C25640D0A000000C3
:106530003401002000C1814001C0804101C0804180
:1065400000C1814001C0804100C1814000C1814043
:1065500001C0804101C0804100C1814000C1814033
:1065600001C0804100C1814001C0804101C0804123
:1065700000C1814001C0804100C1814000C1814013
:1065800001C0804100C1814001C0804101C0804103
:1065900000C1814000C1814001C0804101C08041F3
:1065A00000C1814001C0804100C1814000C18140E3
:1065B00001C0804101C0804100C1814000C18140D3
:1065C00001C0804100C1814001C0804101C08041C3
:1065D00000C1814000C1814001C0804101C08041B3
:1065E00000C1814001C0804100C1814000C18140A3
:1065F00001C0804100C1814001C0804101C0804193
:1066000000C1814001C0804100C1814000C1814082
:1066100001C0804101C0804100C1814000C1814072
:1066200001C0804100C1814001C0804101C0804162
:1066300000C1814000C0C101C30302C2C60607C732
:1066400005C5C404CC0C0DCD0FCFCE0E0ACACB0BA2
:10665000C90908C8D81819D91BDBDA1A1EDEDF1FD2
:10666000DD1D1CDC14D4D515D71716D6D21213D3C2
:1066700011D1D010F03031F133F3F23236F6F73772
:10668000F53534F43CFCFD3DFF3F3EFEFA3A3BFB62
:1066900039F9F83828E8E929EB2B2AEAEE2E2FEF12
:1066A0002DEDEC2CE42425E527E7E62622E2E32382
:1066B000E12120E0A06061A163A3A26266A6A767B2
:1066C000A56564A46CACAD6DAF6F6EAEAA6A6BAB22
:1066D00069A9A86878B8B979BB7B7ABABE7E7FBF52
:1066E0007DBDBC7CB47475B577B7B67672B2B37342
:1066F000B17170B0509091519353529296565797F2
:10670000559594549C5C5D9D5F9F9E5E5A9A9B5BE1
:1067100099595898884849894B8B8A4A4E8E8F4F91
:106720008D4D4C8C44848545874746868242438301
:1067300041818040000303060104060205000305B1
:106740001F1C1F1E1F1E1F1F1E1F1E1F6C67000801
:1067500000000020F4050000280A00084468000832
:10676000F4050020A4330000FC3600081184A24A7E
:1067700004500C010203040607080917EF011CEE80
:10678000EE011C14FA02BC2A6402FFFFFFFFEEEECA
:106790000212FA0312FA0412FA0512EA061203169A
:1067A000B5050D12FFFCFFFF17091115256F1283A8
:1067B0003AA3AA4329D269D60552020406081AAAA6
:1067C0000101200033FF2F7379732F6870386F51E8
:1067D000684D5A4A36372F446576696365312F74A0
:1067E00068696E672F6576656E742F70726F70655D
:1067F0007274792F706F737401CF28232F7379739C
:106800002F6870386F51684D5A4A36372F44657675
:10681000696365312F7468696E672F7365720F182D
:106820000A2F70726F70657274791102FF7401DC47
:1068300052014A0207C91599101A0313045509D4C5
:046840000C00000048
:04000005080000ED02
:00000001FF
